:100000000C94A3000C94CB000C94CB000C94CB006C
:100010000C94CB000C94CB000C94CB000C94CB0034
:100020000C94CB000C94CB000C94CB000C94CB0024
:100030000C94CB000C94CB000C94CB000C94CB0014
:100040000C94CA050C94CB000C94CB000C94CB0000
:100050000C94CB000C94CB000C94CB000C94CB00F4
:100060000C94CB000C94CB0007634236B79BD8A707
:100070001A39685618AEBAAB558C1D3CB7CC5763CD
:10008000BD6DEDFD753EF6177231BF000000803F7B
:1000900008000000BE922449123EABAAAA2ABECD97
:1000A000CCCC4C3E00000080BEABAAAAAA3E000009
:1000B0000000BF000000803F000000000008417801
:1000C000D3BB4387D1133D190E3CC3BD4282AD2B38
:1000D0003E68EC8276BED98FE1A93E4C80EFFFBE30
:1000E00001C4FF7F3F00000000000000000023006B
:1000F0002600290000000000240027002A0000003C
:100100000000250028002B00040404040404040457
:1001100002020202020203030303030301020408B2
:100120001020408001020408102001020408102061
:1001300000000008000201000003040700000000A6
:1001400000000000490A11241FBECFEFD8E0DEBF37
:10015000CDBF11E0A0E0B1E0EEEEFDE102C0059000
:100160000D92A433B107D9F727E0A4E3B1E001C0B1
:100170001D92A539B207E1F710E0C3EAD0E004C050
:100180002197FE010E94EF0EC23AD107C9F70E94E3
:1001900014060C94F50E0C940000CF92DF92EF92AF
:1001A000FF920F931F93CF93DF938C01EB01E1E953
:1001B000F7E080819181A281B3816C017D012DE006
:1001C000CC0CDD1CEE1CFF1C2A95D1F7C826D926C5
:1001D000EA26FB26D701C60131E1B695A79597958A
:1001E00087953A95D1F7C826D926EA26FB26D70166
:1001F000C60145E0880F991FAA1FBB1F4A95D1F77A
:10020000C826D926EA26FB26C082D182E282F38262
:1002100099278F2D7E2D6D2D0E94460C20E030E019
:1002200040E853E30E94FD0C6B017C01BE01601BA2
:10023000710B072E000C880B990B0E94480C9B0138
:10024000AC01C701B6010E94FD0C0E94100CC80150
:10025000860F971FDF91CF911F910F91FF90EF9025
:10026000DF90CF900895833081F028F4813099F0A9
:100270008230A9F008958730A9F08830C9F0843021
:10028000B1F4809180008F7D03C0809180008F77D2
:1002900080938000089584B58F7784BD089584B5D8
:1002A0008F7DFBCF8091B0008F778093B000089551
:1002B0008091B0008F7DF9CF1F93CF93DF93E3E35D
:1002C000F1E09491EFE1F1E0D491EBE0F1E0C49141
:1002D000CC23B9F0182F992319F0892F0E943301EC
:1002E000EC2FF0E0EE0FFF1FE250FF4FA591B4910D
:1002F0008FB7F894EC91111108C0D095DE23DC93F0
:100300008FBFDF91CF911F910895DE2BF8CFCF9350
:10031000DF9390E0FC01E45EFE4F2491885F9E4FE6
:10032000FC0184918823C9F090E0880F991FFC019B
:10033000EC50FF4FA591B491FC01E250FF4FC591E5
:10034000D49161110DC09FB7F8948C9120958223B0
:100350008C938881282328839FBFDF91CF910895B4
:10036000623051F49FB7F8943C91822F809583239B
:100370008C93E8812E2BEFCF8FB7F894EC912E2B36
:100380002C938FBFEACF8E50806480937C00809145
:100390007A00806480937A0080917A0086FDFCCF99
:1003A000809178009091790008953FB7F8948091FA
:1003B0004E0190914F01A0915001B091510126B58D
:1003C000A89B05C02F3F19F00196A11DB11D3FBF8D
:1003D000BA2FA92F982F8827BC01CD01620F711D5C
:1003E000811D911D42E0660F771F881F991F4A9556
:1003F000D1F708952F923F924F925F926F927F9222
:100400008F929F92AF92BF92CF92DF92EF92FF9224
:100410000F931F93CF93DF93CDB7DEB7CA59D1099E
:100420000FB6F894DEBF0FBECDBF81E00E945C0125
:1004300081E080933C012FB7F89480914A0190911C
:100440004B01A0914C01B0914D012FBF8093380119
:1004500090933901A0933A01B0933B0180E10E944F
:10046000C3019C01990F440B550B211584E03807FB
:100470004105510524F02FEF33E040E050E057FFF5
:1004800003C020E030E0A901A9E0B0E00E94F00A3A
:100490002FEF33E040E050E00E94D10A2D5F3F4F44
:1004A0004F4F5F4F190185E10E94C3016C0184E148
:1004B0000E94C3010D2C000CEE08FF0864E1CC0C77
:1004C000DD1CEE1CFF1C6A95D1F7092E000CAA0B4F
:1004D000BB0B7AE0880F991FAA1FBB1F7A95D1F733
:1004E000C826D926EA26FB260E94D501C616D706BD
:1004F000E806F90609F463C1C626D726E826F926D8
:10050000C0929107D0929207E0929307F0929407DD
:10051000A2E5B1E0C757DF4FB983A883C958D040DF
:10052000F1013197C957DF4FF983E883C758D040AD
:10053000EE0FFF1FEE0FFF1FCF56DF4FF983E8834B
:10054000C159D0406E01F1E4CF0ED11CF12CE12C49
:10055000860168EE73E090E080E00E94CD00BC016F
:10056000990F880B990B0E94480C20E030E04AE775
:1005700054E40E949E0BD6016D937D938D939D93C1
:100580006D01BFEFEB1AFB0AE214F30414F3B1019F
:1005900090E080E00E94CD00880F991F880F991F7E
:1005A000F801E80FF91F1082118212821382B10143
:1005B00090E080E00E94CD00880F991F880F991F5E
:1005C000F801E80FF91F80E090E0A0E8BFE3808326
:1005D0009183A283B383DE0111967D015D01412CDD
:1005E000512C3201D12CC12C4D0168EC70E082E31A
:1005F00090E00E94CD00BC01990F880B990B0E94DE
:10060000480C20E030E04AE754E40E949E0B9B0136
:10061000AC01C301B2010E942D0B2B013C01F5017D
:1006200041925192619271925F01FFEFCF1ADF0AFE
:10063000C214D304D4F220E030E0A9010E94990B47
:10064000181634F0412C512C80E8682E8FE3782E58
:10065000D12CC12CD7016D917D918D919D917D0102
:100660005D01B4E0AB1AB108A30192010E949E0B98
:10067000F5016083718382839383FFEFCF1ADF0AD2
:10068000C214D3043CF3F80180819181A281B3812B
:10069000CF56DF4FE881F981C159D040E00FF11FFB
:1006A00080839183A283B383CF56DF4FE881F981A2
:1006B000C159D040E80DF91D80E090E0A0E8BFE30B
:1006C00080839183A283B383C957DF4F6881798187
:1006D000C758D04090E080E00E94CD00C157DF4F66
:1006E00099838883CF58D04060E570E080EB9FEF1E
:1006F0000E94CD00BC01990F880B990B0E94480CF9
:1007000020E030E048EC52E40E949E0BCB56DF4FD5
:10071000688379838A839B83C559D040CB57DF4F49
:1007200019821882C558D040C157DF4F88819981FE
:10073000CF58D040880F991F880F991FA1E4B0E0CF
:10074000AC0FBD1FA80FB91FC756DF4FB983A883D1
:10075000C959D040CB57DF4FE881F981C558D04007
:10076000BF01FF0F880B990B0E94480C20E030E07E
:100770004FE753E40E949E0B4B015C017E01F5E0C4
:10078000EF0EF11C10E000E0C8010196CF57DF4FDB
:1007900099838883C158D040D7012D913D914D91C7
:1007A0005D917D01C501B4010E94F80C18167CF022
:1007B000CF57DF4F19830883C158D04017C05EEE72
:1007C000C52EDD24DA9450ECE52EF12C99CECF57CE
:1007D000DF4F08811981C158D040C957DF4F2881A8
:1007E0003981C758D0400217130774F2CF57DF4F33
:1007F00008811981C158D0400F5F1F4F02151305A2
:1008000034F0C957DF4F08811981C758D040CF57FE
:10081000DF4FE881F981C158D040EE0FFF1FEE0F86
:10082000FF1FCD56DF4FF983E883C359D040E1E085
:10083000F0E0EC0FFD1FCD56DF4F28813981C35901
:10084000D040E20FF31F4080518062807380000F20
:10085000111F000F111FE1E0F0E0EC0FFD1FE00F92
:10086000F11FA301920160817181828193810E94B5
:100870002C0B6B017C0120E030E0A9010E94990B58
:10088000882309F458C1A3019201C501B4010E9453
:100890002C0BA70196010E949E0B6B017C01E1E4E9
:1008A000F0E0EC0FFD1FE00FF11F80819181A2812C
:1008B000B381C557DF4F88839983AA83BB83CB5805
:1008C000D040C157DF4FA881B981CF58D040CF5712
:1008D000DF4FE881F981C158D040AE17BF0709F05A
:1008E00032C1C756DF4FA881B981C959D0408D9117
:1008F0009D910D90BC91A02DCF57DF4F8883998398
:10090000AA83BB83C158D040C557DF4F28813981A6
:100910004A815B81CB58D040BC01CD010E942D0B98
:1009200020E030E040E05FE30E94FD0CCB56DF4F5B
:10093000288139814A815B81C559D0400E942D0BA5
:100940004B015C0120E030E0A9010E94990B87FD7A
:10095000F6C020E030E040E85FE3C501B4010E944A
:10096000F80C181634F4812C912CE0E8AE2EEFE34D
:10097000BE2EA701960160E070E080E89FE30E9430
:100980002C0B2B013C01AC019B010E942D0BA701FC
:1009900096010E94FD0CA50194010E94FD0C4B01E3
:1009A0005C01A3019201C301B2010E94FD0CCF576B
:1009B000DF4F288139814A815B81C158D0400E9434
:1009C000FD0C9B01AC01C501B4010E942D0B4B0134
:1009D0005C01A7019601C701B6010E94FD0CC55735
:1009E000DF4F288139814A815B81CB58D0400E94FA
:1009F000FD0C9B01AC01C501B4010E942D0B6B01E4
:100A00007C0120E030E0A9010E94990B87FDBEC067
:100A100020E030E040E85FE3C701B6010E94F80C37
:100A2000181634F4C12CD12C70E8E72E7FE3F72E92
:100A3000CB57DF4F08811981C558D040000F111FD7
:100A4000C757DF4F88819981C958D040080F191FB7
:100A500020E03FEF4FE757E4C701B6010E94FD0CCD
:100A60000E94170CD8016D937C93CB57DF4FE88120
:100A7000F981C558D0403196CB57DF4FF983E883D1
:100A8000C558D040E115F14009F064CEC757DF4F9B
:100A900088819981C958D0409E5FC757DF4F99839D
:100AA0008883C958D0408255974009F04BCD82E5E4
:100AB00097E02AE637E04DE0BE016F5F7F4FC12C23
:100AC000D12C50E8E52E5FE3F52EFC011192119236
:100AD00011921192CF01DB01E42F1D92EA95E9F703
:100AE000CA82DB82EC82FD82FB01D901542F019086
:100AF0000D925A95E1F7235F3F4FF7E08E359F0740
:100B000021F7C656DF4F0FB6F894DEBF0FBECDBF3C
:100B1000DF91CF911F910F91FF90EF90DF90CF90D9
:100B2000BF90AF909F908F907F906F905F904F900D
:100B30003F902F900895C12CD12C7601B0CE812CFE
:100B4000912C540116CFE1E4F0E0EC0FFD1FCD56DF
:100B5000DF4F28813981C359D040E20FF31F8080D5
:100B60009180A280B380A5019401C557DF4F6881B1
:100B700079818A819B81CB58D0400E942C0BA701A0
:100B800096010E94FD0CA501940137CFC12CD12CF8
:100B900076014ECF1F920F920FB60F9211242F9312
:100BA0003F938F939F93AF93BF9380914A0190910E
:100BB0004B01A0914C01B0914D013091490123E0CE
:100BC000230F2D3758F50196A11DB11D2093490122
:100BD00080934A0190934B01A0934C01B0934D0137
:100BE00080914E0190914F01A0915001B09151011F
:100BF0000196A11DB11D80934E0190934F01A093CA
:100C00005001B0935101BF91AF919F918F913F914E
:100C10002F910F900FBE0F901F90189526E8230F6D
:100C20000296A11DB11DD2CFCF93DF93CDB7DEB712
:100C300062970FB6F894DEBF0FBECDBF789484B52F
:100C4000826084BD84B5816084BD85B5826085BDC8
:100C500085B5816085BD80916E00816080936E0056
:100C60001092810080918100826080938100809148
:100C700081008160809381008091800081608093F9
:100C800080008091B10084608093B1008091B000B9
:100C900081608093B00080917A00846080937A00B4
:100CA00080917A00826080937A0080917A008160DE
:100CB00080937A0080917A00806880937A00109205
:100CC000C10060E08EE00E94870160E08FE00E943A
:100CD000870160E080E10E94870160E081E10E947D
:100CE000870162E084E00E94870161E083E00E9466
:100CF000870161E089E00E94870161E08AE00E944B
:100D0000870161E08BE00E94870181EA8093800087
:100D100089E08093810083E88093B00082E0809333
:100D2000B10020E830E030938900209388003093B0
:100D30008B0020938A0080E88093B3000E94FA0120
:100D40008FB7F894C0904A01D0904B01E0904C01CD
:100D5000F0904D018FBFE4E3F1E08491E0E2F1E037
:100D6000F491F983ECE0F1E0F491FB83FF2389F047
:100D700081110E9433012B81E22FF0E0EE0FFF1F63
:100D8000E651FF4FA591B4918C913981382381E0D0
:100D900009F480E0109247011092480190914601B9
:100DA000891751F080934601C0924101D0924201CF
:100DB000E0924301F09244018091410190914201FF
:100DC000A0914301B0914401C81AD90AEA0AFB0A6A
:100DD00080913D0190913E01A0913F01B091400171
:100DE0008C159D05AE05BF05B0F49091450180912D
:100DF0004601981781F080934501911103C021E0CD
:100E0000813009F020E020934701913009F48111ED
:100E100090E0909348018091480181110E94FA016D
:100E200080913C01882309F12FB7F89480914A0101
:100E300090914B01A0914C01B0914D012FBF409179
:100E400038015091390160913A0170913B01841B46
:100E5000950BA60BB70B893C9105A105B10528F0B0
:100E600080E00E945C0110923C018EE00E94C30170
:100E7000BC01990F880B990B0E94480C20E030ECC4
:100E80004FE754E40E949E0B6B017C018FE00E94AF
:100E9000C301BC01990F880B990B0E94480C20E0FC
:100EA00030EC4FE754E40E949E0B6B837C838D8370
:100EB0009E8380E10E94C30120E030E0A901C701C8
:100EC000B6010E94990B87FD96C120E030E040E812
:100ED0005FE3C701B6010E94F80C18160CF48FC12D
:100EE000A701960160E070E086E993E40E946A0D34
:100EF0002AE037ED43E25CE30E94FD0C2B013C014C
:100F000020E030E0A9016B817C818D819E810E946F
:100F1000990B87FD7BC120E030E040E85FE36B8107
:100F20007C818D819E810E94F80C18160CF473C18F
:100F300081E10E94C3019C01990F440B550B2115BF
:100F400094E039074105510524F02FEF33E040E0EC
:100F500050E057FF03C020E030E0A901A8EEB3E065
:100F60000E94F00A2FEF33E040E050E00E94D10AE7
:100F7000CA01B9010E94480C20E030E04AE754E47D
:100F80000E949E0B4B015C010E94D5016B017C010C
:100F90008091340190913501A0913601B0913701D3
:100FA000A7019601281B390B4A0B5B0BCA01B9013B
:100FB0000E94460C20E034E244E759E40E949E0B74
:100FC0006F83788789879A8720E030E0A9010E94A3
:100FD000990B181644F08FE692E1A3E8BAE38F83E9
:100FE0009887A987BA87C0923401D0923501E092E0
:100FF0003601F0923701A3019201C501B4010E94AC
:101000002D0B4B015C0120E030E0A9010E94990BFF
:1010100087FD0AC120E030E040E251E4C501B4019F
:101020000E94F80C181634F4812C912C40E2A42E66
:1010300041E4B42E0AE617E032E5232E37E0332EE2
:10104000A7E2B1E0BA83A9831C861B86F8018081E0
:10105000811172C060E177E290E080E00E94CD00F3
:10106000BC01990F880B990B0E94480C6B017C0105
:1010700020E030E040EA50E46B817C818D819E81EC
:101080000E94FD0C9B01AC01C701B6010E94990BA7
:1010900087FF4DC0E1E0D801EC9362E370E08AE0A5
:1010A00090E00E94CD00BC01990F880B990B0E9423
:1010B000480C20E030E048EC52E40E949E0BD8013E
:1010C00011966D937D938D939C93149768EB7BE0C1
:1010D00088EC90E00E94CD00BC01990F880B990B21
:1010E0000E94480C20E030E048E454E40E942D0BBC
:1010F0006B017C012DEC3CEC4CEC5DE3C501B401D3
:101100000E942D0B9B01AC01C701B6010E949E0BF2
:101110002FE632E143E85AE30E94FD0CF8016583B3
:101120007683878390871186128613861486F8014A
:101130008081882309F4A4C1D80119962D913D918D
:101140004D915C911C976F81788589859A850E9465
:101150002D0BF801618772878387948725813681FB
:10116000478150850E94F80CE981FA81349618165F
:101170000CF074C1D8011C92A981BA812D913D91C6
:101180004D915C91FA83E983C501B4010E94FD0C85
:1011900020E030E040E853E40E94FD0C2F813885C8
:1011A00049855A850E94FD0C9B01AC01F1016081CB
:1011B0007181828193810E942D0BD1016D937D936A
:1011C0008D939C931397F101C080D180E280F380CE
:1011D00020E030E040E853E4C701B6010E94F80C7B
:1011E00087FD26C020E030E040E853E4C701B601A7
:1011F0000E942C0BE2CFC12CD12C760171CEC12CD8
:10120000D12C50E8E52E5FE3F52E6ACE1B821C82BE
:101210001D821E828DCE80E090E0A0E8BFE38B832C
:101220009C83AD83BE8384CE812C912C540102CF4C
:10123000F101C080D180E280F38020E030E0A9019C
:10124000C701B6010E94990B87FF0FC020E030E074
:1012500040E853E4C701B6010E942D0BD1016D9304
:101260007D938D939C931397E3CFC701B6010E94A2
:10127000100C7E876D876F3F710529F024F02FEFEA
:1012800030E03E872D874D855E855A8B498B57FF11
:1012900002C01A8A198A69887A885FEF651A750A06
:1012A000611481E0780611F4712C612CAB85BC854A
:1012B0005A2E4424E989FA89E40DF51DEE0FFF1F2B
:1012C000EE5AFE4F6081718190E080E00E94460CF2
:1012D00020E830E040E857E30E94FD0C6D877E87F0
:1012E0008F87988BF201E60DF71DEE0FFF1FEE5A68
:1012F000FE4F6081718190E080E00E94460C20E802
:1013000030E040E857E30E94FD0C2D853E854F8577
:1013100058890E942C0B2B013C01E989FA89BF01F5
:10132000FF0F880B990B0E94480C9B01AC01C70171
:10133000B6010E942C0B9B01AC01C301B2010E94BB
:10134000FD0C2D853E854F8558890E942D0B2DEC77
:101350003CEC4CEC5DE30E94FD0C6B017C0126E64D
:1013600036E646E65FE3D1011C966D917D918D9145
:101370009C911F970E94FD0C9B01AC01C701B60117
:101380000E942D0BF10164877587868797872B85CF
:101390003C852F5F3F4F3C872B87035F1F4F34E017
:1013A000230E311C4B855C854330510509F04ECE30
:1013B00020E030E04FE753E460915E0770915F07F3
:1013C00080916007909161070E94FD0C20E030E061
:1013D00040E05FE30E942D0B0E94170C70E07093B9
:1013E00089006093880020E030E04FE753E460918B
:1013F00062077091630780916407909165070E946E
:10140000FD0C20E030E040E05FE30E942D0B0E94E5
:10141000170C70E070938B0060938A0020E030E03E
:101420004FE753E460916607709167078091680702
:10143000909169070E94FD0C20E030E040E05FE3FE
:101440000E942D0B0E94170C6093B30080E090E087
:10145000892B09F475CC0E94000072CCA981BA8155
:101460006D917D918D919C91FA83E983A501940101
:101470000E94FD0CF801218132814381548186CE86
:10148000A981BA812D913D914D915D91BA83A98336
:101490007BCE8F929F92AF92BF92CF92DF92EF92CC
:1014A000FF92CF93DF93CDB7DEB72D970FB6F894A9
:1014B000DEBF0FBECDBF87E2E0E0F1E0AAE6B7E015
:1014C00001900D928A95E1F78EEE9FEFA0ECB0E0CF
:1014D0008093910790939207A0939307B0939407FA
:1014E00082E597E02AE637E0812C912CA12C4FE38E
:1014F000B42E4DE0BE016F5F7F4FC12CD12C50E860
:10150000E52E5FE3F52EFC011192119211921192DA
:10151000CF0180869186A286B386FB01542F11925B
:101520005A95E9F7CA82DB82EC82FD82FB01D90180
:10153000542F01900D925A95E1F7235F3F4FE7E05A
:101540008E359E0701F782E390E0A0E0B0E0809343
:101550003D0190933E01A0933F01B0934001109252
:10156000410110924201109243011092440181E026
:1015700080934501809346011092470110924801E3
:101580002D960FB6F894DEBF0FBECDBFDF91CF9181
:10159000FF90EF90DF90CF90BF90AF909F908F9093
:1015A0000895052E97FB1EF400940E94E80A57FD4B
:1015B00007D00E94FB0A07FC03D04EF40C94E80A03
:1015C00050954095309521953F4F4F4F5F4F08956F
:1015D00090958095709561957F4F8F4F9F4F08959F
:1015E0000E941D0BA59F900DB49F900DA49F800D90
:1015F000911D11240895A1E21A2EAA1BBB1BFD0107
:101600000DC0AA1FBB1FEE1FFF1FA217B307E407E1
:10161000F50720F0A21BB30BE40BF50B661F771F39
:10162000881F991F1A9469F7609570958095909519
:101630009B01AC01BD01CF010895A29FB001B39FF2
:10164000C001A39F700D811D1124911DB29F700DCB
:10165000811D1124911D08955058BB27AA270E946F
:10166000440B0C94BE0C0E94B00C38F00E94B70CD6
:1016700020F039F49F3F19F426F40C94AD0C0EF4CD
:10168000E095E7FB0C94A70CE92F0E94CF0C58F3D0
:10169000BA17620773078407950720F079F4A6F557
:1016A0000C94F10C0EF4E0950B2EBA2FA02D0B012B
:1016B000B90190010C01CA01A0011124FF27591B97
:1016C00099F0593F50F4503E68F11A16F040A22F9D
:1016D000232F342F4427585FF3CF4695379527950E
:1016E000A795F0405395C9F77EF41F16BA0B620B0D
:1016F000730B840BBAF09150A1F0FF0FBB1F661F54
:10170000771F881FC2F70EC0BA0F621F731F841F96
:1017100048F4879577956795B795F7959E3F08F0BC
:10172000B0CF9395880F08F09927EE0F979587957E
:1017300008950E94830C08F481E008950E94B20B82
:101740000C94BE0C0E94B70C58F00E94B00C40F0F4
:1017500029F45F3F29F00C94A70C51110C94F20C62
:101760000C94AD0C0E94CF0C68F39923B1F3552370
:1017700091F3951B550BBB27AA27621773078407A4
:1017800038F09F5F5F4F220F331F441FAA1FA9F33A
:1017900035D00E2E3AF0E0E832D091505040E69528
:1017A000001CCAF72BD0FE2F29D0660F771F881F89
:1017B000BB1F261737074807AB07B0E809F0BB0B7C
:1017C000802DBF01FF2793585F4F3AF09E3F510590
:1017D00078F00C94A70C0C94F20C5F3FE4F3983E65
:1017E000D4F3869577956795B795F7959F5FC9F779
:1017F000880F911D9695879597F90895E1E0660FFA
:10180000771F881FBB1F621773078407BA0720F072
:10181000621B730B840BBA0BEE1F88F7E0950895DB
:101820000E94170C6894B1110C94F20C08950E9458
:10183000D70C88F09F5798F0B92F9927B751B0F07F
:10184000E1F0660F771F881F991F1AF0BA95C9F744
:1018500014C0B13091F00E94F10CB1E008950C94E5
:10186000F10C672F782F8827B85F39F0B93FCCF398
:10187000869577956795B395D9F73EF490958095C1
:10188000709561957F4F8F4F9F4F0895E89409C0E1
:1018900097FB3EF490958095709561957F4F8F4FA3
:1018A0009F4F9923A9F0F92F96E9BB279395F695B9
:1018B000879577956795B795F111F8CFFAF4BB0F37
:1018C00011F460FF1BC06F5F7F4F8F4F9F4F16C09B
:1018D000882311F096E911C0772321F09EE8872F25
:1018E000762F05C0662371F096E8862F70E060E0E1
:1018F0002AF09A95660F771F881FDAF7880F96955A
:10190000879597F90895990F0008550FAA0BE0E8FD
:10191000FEEF16161706E807F907C0F012161306B1
:10192000E407F50798F0621B730B840B950B39F4F1
:101930000A2661F0232B242B252B21F408950A2657
:1019400009F4A140A6958FEF811D811D089597F997
:101950009F6780E870E060E008959FEF80EC089555
:1019600000240A941616170618060906089500247E
:101970000A9412161306140605060895092E0394F8
:10198000000C11F4882352F0BB0F40F4BF2B11F46C
:1019900060FF04C06F5F7F4F8F4F9F4F089557FDCB
:1019A0009058440F551F59F05F3F71F04795880FCD
:1019B00097FB991F61F09F3F79F087950895121664
:1019C00013061406551FF2CF4695F1DF08C0161610
:1019D00017061806991FF1CF8695710561050894C1
:1019E0000895E894BB2766277727CB0197F90895D8
:1019F0000E94830C08F48FEF08950E94100D0C9440
:101A0000BE0C0E94B00C38F00E94B70C20F0952359
:101A100011F00C94A70C0C94AD0C11240C94F20C46
:101A20000E94CF0C70F3959FC1F3950F50E0551FA6
:101A3000629FF001729FBB27F00DB11D639FAA2723
:101A4000F00DB11DAA1F649F6627B00DA11D661F72
:101A5000829F2227B00DA11D621F739FB00DA11D93
:101A6000621F839FA00D611D221F749F3327A00D4D
:101A7000611D231F849F600D211D822F762F6A2FE9
:101A800011249F5750409AF0F1F088234AF0EE0F4E
:101A9000FF1FBB1F661F771F881F91505040A9F77B
:101AA0009E3F510580F00C94A70C0C94F20C5F3F04
:101AB000E4F3983ED4F3869577956795B795F795B7
:101AC000E7959F5FC1F7FE2B880F911D969587952F
:101AD00097F90895FA01EE0FFF1F309621053105A1
:101AE000A1F16115710561F48038BFE39B0749F1ED
:101AF00068949038810561F08038BFEF9B0741F012
:101B000099234AF5FF3FE1053105210519F1E894D4
:101B10000894E795D901AA2329F4AB2FBE2FF85FCB
:101B2000D0F310C0FF5F70F4A695E0F7F73950F0DE
:101B300019F0FF3A38F49F779F930DD00F9007FC70
:101B40009058089546F00C94AD0C60E070E080E889
:101B50009FE308954FE79F775F934F933F932F93B2
:101B60000E94650E2F913F914F915F910E94FD0C55
:101B70000C94C20D29F416F00C94A70C0C94F10CE3
:101B80000C94AD0C0E94D70CA8F39638A0F707F878
:101B90000F92E8942BE33AEA48EB5FE70E94130DBB
:101BA0000F920F920F924DB75EB70F920E94AD0E3B
:101BB000E8E6F0E00E94F40D4F915F91EF91FF9104
:101BC000E595EE1FFF1F49F0FE57E0684427EE0F32
:101BD000441FFA95E1F74195550B0E94270E0F908F
:101BE00007FE0C941B0E0895DF93CF931F930F9362
:101BF000FF92EF92DF927B018C01689406C0DA2E8F
:101C0000EF010E94100DFE01E894A59125913591F8
:101C100045915591A6F3EF010E94440BFE019701F7
:101C2000A801DA9469F7DF90EF90FF900F911F9170
:101C3000CF91DF9108959B01AC0160E070E080E8F6
:101C40009FE30C949E0B0C94A70C0C94E10E0E9445
:101C5000D70CD8F39923C9F3940F511DA3F39150D6
:101C6000504094F059F0882332F0660F771F881F98
:101C700091505040C1F79E3F51052CF7880F911DA0
:101C80009695879597F908955F3FACF0983E9CF044
:101C9000BB27869577956795B79508F4B1609395BE
:101CA000C1F7BB0F58F711F460FFE8CF6F5F7F4FAC
:101CB0008F4F9F4FE3CF0C94F20C16F00C94E10E73
:101CC0000C94AD0C68940C94A70C0E94D70CA8F34C
:101CD0009923C1F3AEF3DF93CF931F930F93FF923A
:101CE000C92FDD2788232AF02197660F771F881FC9
:101CF000DAF720E030E040E85FEB9FE3883920F03E
:101D0000803E38F021968F770E942D0BE0E9F0E0BD
:101D100004C00E942D0BEDEBF0E00E94F40D8B014E
:101D2000BE01EC01FB2E6F5771097595771F880B6B
:101D3000990B0E94480C28E132E741E35FE30E94DF
:101D4000100DAF2D9801AE01FF900F911F91CF9113
:101D5000DF910E94440B0C94BE0CFA01DC01AA0F27
:101D6000BB1F9B01AC01BF5728F422273327442710
:101D7000507820C0B75190F4AB2F0024469537958A
:101D80002795011CA395D2F3002071F0220F331F79
:101D9000441FB395DAF30ED00C942C0B613071050F
:101DA000A0E88A07B94630F49B01AC016627772783
:101DB00088279078309621F02083318342835383A3
:101DC00008959F3F31F0915020F48795779567955E
:101DD000B795880F911D9695879597F90895EE0F01
:0E1DE000FF1F0590F491E02D0994F894FFCFB9
:101DEE00000000803F000000000000000000000026
:101DFE00803F0000000000000000000000803F0057
:101E0E00000000000000006666663F0000803FCDC7
:041E1E00CC8C3F0029
:00000001FF
